:020000040801F1
:10000000104200209D010108A5010108A701010877
:10001000A9010108AB010108AD01010800000000C1
:10002000000000000000000000000000AF01010817
:10003000B101010800000000B3010108E90B01084B
:10004000B7010108B7010108B7010108B7010108AC
:10005000B7010108B7010108B7010108B70101089C
:10006000B7010108B7010108B7010108B70101088C
:10007000B7010108B7010108B7010108B70101087C
:10008000B7010108B7010108B7010108B70101086C
:10009000B7010108B7010108B7010108B70101085C
:1000A000B7010108B7010108B7010108B70101084C
:1000B000B7010108B7010108B7010108B70101083C
:1000C000B7010108B7010108B7010108B70101082C
:1000D000B7010108B7010108B7010108B70101081C
:1000E000B7010108B7010108B7010108B70101080C
:1000F000B7010108B7010108B7010108B7010108FC
:10010000B7010108B7010108B7010108B7010108EB
:10011000B7010108B7010108B7010108B7010108DB
:10012000B7010108B7010108B7010108B7010108CB
:10013000B7010108B7010108B7010108B7010108BB
:10014000B7010108B7010108B7010108B7010108AB
:10015000B7010108B7010108B7010108B70101089B
:10016000B7010108B7010108B7010108B70101088B
:10017000B7010108B7010108B7010108000000003C
:10018000B7010108B7010108DFF80CD000F04AF808
:1001900000480047D9110108104200200648804756
:1001A00006480047FEE7FEE7FEE7FEE7FEE7FEE75C
:1001B000FEE7FEE7FEE7FEE7650C0108890101089E
:1001C0002DE9F05F0546002092469B46884606468C
:1001D000814640241BE0284641464746224600F01F
:1001E00042F853465A46C01A914110D31146184658
:1001F000224600F029F82D1A67EB01084F462246E7
:100200000120002100F020F817EB00094E41201ECC
:10021000A4F10104DFDC484631462A464346BDE8E6
:10022000F09F0000064C074D06E0E06840F0010337
:1002300094E8070098471034AC42F6D3FFF7A8FFC4
:10024000E012010800130108202A04DB203A00FA1A
:1002500002F1002070479140C2F1200320FA03F31D
:10026000194390407047202A04DB203A21FA02F01B
:100270000021704721FA02F3D040C2F120029140E0
:1002800008431946704700002DE9F84FDFF89491B4
:10029000002209F1040A0AF1040B4FF00F080BF1D8
:1002A000040E01260B6896403340B34271D14C686E
:1002B000022C01D0122C11D1D40800EB84073D6A26
:1002C0005407E40E08FA04FC25EA0C05D1F810C026
:1002D0000CFA04FC4CEA050CC7F820C0076854006F
:1002E000032591F804C0A5400CF0030CAF430CFAB1
:1002F00004FC4CEA070CC0F800C04F68012F05D081
:10030000022F03D0112F01D0122F11D18768D1F8FD
:100310000CC0AF430CFA04FC4CEA070CC0F808C050
:100320004768B7430E79C6F3001696403E434660D1
:10033000C668AE438D68A5403543C5604C68E4008F
:100340006AD5394C256845F480452560246822F03B
:10035000030504F480440094344C2544D5F808780F
:100360009407260F08FA06F4A743314CA04201D1A6
:10037000002429E02F4CA04201D1012424E02E4C7E
:10038000A04201D102241FE02C4CA04202D1032440
:100390001AE041E02A4CA04201D1042414E0294C87
:1003A000A04201D105240FE0274CA04201D1062430
:1003B0000AE0264CA04201D1072405E0244CA042CB
:1003C00001D1082400E00924B4403C43C5F80848A2
:1003D000D9F800404D464E689C43F60300D51C43B7
:1003E0002C60DAF8004055464E689C43B60300D5B1
:1003F0001C432C60DBF800405D464E689C43F602CF
:1004000000D51C432C60DEF8004075464E689C43C6
:10041000B60200D51C432C60521C102AFFF441AFD9
:10042000BDE8F88F003C01404438024000300140F4
:10043000000002400004024000080240000C02409C
:10044000001002400014024000180240001C02404C
:1004500000200240014800687047000004000020AE
:1004600002480168491C0160704700000400002038
:100470000B4810B5016841F400710160016841F456
:1004800080610160016841F480710160032000F027
:100490005DF8002000F006F800F015F8002010BD0F
:1004A000003C024010B5044600F062F84FF47A7147
:1004B000B0FBF1F000F075FA00222146501E00F06A
:1004C00025F8002010BD10B5032000F03FF80022F1
:1004D00011466FF00B0000F019F8002211466FF082
:1004E0000A0000F013F8002211466FF0090000F036
:1004F0000DF800221146101F00F008F80022BDE898
:1005000010401146501E00F001B80000F0B40E4B30
:100510001B68C3F30223C3F10704042C00D904248D
:100520001D1D072D01D2002300E0DB1E012606FA67
:1005300004F56D1E0D409D409E40761E164045EA16
:100540000601F0BC00F040BB0CED00E0064A00F0F4
:10055000070110684FF6FF03184040EA01200349E5
:1005600008431060704700000CED00E00000FA0541
:1005700010B500F043F808490968F02292FAA2F297
:1005800001F0F001B2FA82F2D140044A515CC84055
:100590000349086010BD000008380240D01201086D
:1005A0000800002010B5FFF7E3FF074909684FF482
:1005B000E05292FAA2F201F4E051B2FA82F2D14092
:1005C000024A515CC84010BD08380240D0120108F0
:1005D00010B5FFF7CDFF074909684FF4604292FA62
:1005E000A2F201F46041B2FA82F2D140024A515CB7
:1005F000C84010BD08380240D012010830B5194873
:10060000006810F00C01184812D0184C04290ED0C4
:1006100008290DD1134A121F1168136801F03F0118
:100620005D0247F6C07304D5B4FBF1F003E0204649
:1006300030BDB0FBF1F01168194093FAA3F3B3FA9F
:1006400083F3D940484311684FF4403292FAA2F242
:1006500001F44031B2FA82F2D140491C4900B0FBAA
:10066000F1F030BD083802400024F40040787D01EC
:100670002DE9F84F04460078DFF8F8A2BE4DC00718
:100680004FF0000646D0DAF800105046C1F3810161
:10069000012908D00068C0F3810002280AD1281D72
:1006A0000068400206D52868800333D560680028BA
:1006B00071D02FE0DFF8C08208F1020888F80060EE
:1006C000FFF7C8FE074604E0FFF7C4FEC01B64281E
:1006D0007AD828688003F7D4207988F80000606809
:1006E00060B1FFF7B7FE074604E0FFF7B3FEC01B9B
:1006F0006428EDD828688003F7D50BE0FFF7AAFE41
:10070000074604E0FFF7A6FEC01B6428E0D828686F
:100710008003F7D42078DFF86482800744D5DAF8C4
:100720000010504611F00C0F4FF0F80909D0006886
:10073000C0F3810002280BD18E48001F00684002E0
:1007400006D42868800714D5E068012823D110E07A
:10075000E068D0B10120C8F80000FFF77BFE074633
:1007600004E0FFF777FEC01B6428B1D82868800733
:10077000F7D5286899FAA9F22169B2FA82F220F035
:10078000F8009140084328600EE0C8F80060FFF7C9
:1007900061FE074605E0EAE0FFF75CFEC01B642847
:1007A00012D828688007F7D42078000725D5DFF80D
:1007B000C4917348616909F16C0981B1012101603B
:1007C000FFF748FE074605E07EE0FFF743FEC01B4B
:1007D000642879D8D9F800008007F6D50DE00660C6
:1007E000FFF738FE074604E0FFF734FEC01B64281D
:1007F0006AD8D9F800008007F6D42078400753D58E
:100800005C483830016841F0805101600068DFF8D1
:10081000749100F080500090D9F8001041F480717C
:10082000C9F80010FFF716FE074604E0FFF712FEB6
:10083000C01B642848D8D9F80000C005F6D5DFF8F9
:1008400034B10BF1680B8BF80060FFF703FE07462D
:1008500041F2883904E0FFF7FDFDC11B49457ED810
:10086000DBF800008007F6D4207A8BF80000A0683F
:1008700068B1FFF7EFFD074604E0FFF7EBFDC11B92
:1008800049456CD8DBF800008007F6D50CE0FFF78F
:10089000E1FD074604E0FFF7DDFDC11B49455ED8D9
:1008A000DBF800008007F6D4A069E8B3DAF800109E
:1008B000C1F3810102295AD0022806D0C8F860602D
:1008C000FFF7C8FD04464DE049E04746C8F86060C0
:1008D000FFF7C0FD064604E0FFF7BCFD801B64285F
:1008E0003DD828688001F7D4D4E90710014347F6C2
:1008F000C07090FAA0F0626AB0FA80F08240A06AFC
:100900004FF0FF3303EB50004FF4403393FAA3F35F
:10091000B3FA83F39840024311434FF0706292FAA6
:10092000A2F2B2FA82F200E01FE0E06A90400143D6
:100930001048001F016001203866FFF78BFD044658
:1009400004E0FFF787FD001B642808D828688001B1
:10095000F7D50AE0FFF77EFD001B642802D90320CB
:10096000BDE8F88F28688001F4D40020F8E7012062
:10097000F6E7000008380240003802400000474215
:10098000800E4742007000404FF0E02104280869C3
:1009900003D020F004000861704740F00400FAE73B
:1009A000704710B5401EB0F1807F01D3012010BD0B
:1009B0004FF0E02460610F21601700F005F900207E
:1009C000A06107202061002010BD10B5FFF7E8FFEF
:1009D00010BD70B5040004D094F83900002510B1A2
:1009E00006E0012070BD84F83850204600F020F861
:1009F000022084F839002068C16821F40051C160E8
:100A0000204600F059F92068016921F49041016104
:100A10002068416921F02A0141612068C16841F4E0
:100A20000051C160E563012084F83900002070BDE9
:100A300000B500680E4987B0884217D10D4801689B
:100A400041F4802101600068694600F4802005902F
:100A50004FF440600090022001900120029003209A
:100A60000390072004900448FFF70EFC07B000BD78
:100A70000048004040380240000802402DE9F0479D
:100A8000044690F8390099460D46012801D02228E5
:100A900056D125B31AB394F83800012850D0012656
:100AA00084F838600027E76394F83900222819D0C9
:100AB000122084F83900A284E2844FF48058E08C3C
:100AC0004B46401EE084A0684FF0000240454FF0C6
:100AD0008001204613D100F0A9F908BB04E00120F1
:100AE000BDE8F0873220E4E728882168C0F30800D9
:100AF0004860206908B16D1C08E0AD1C06E000F0FC
:100B000095F968B9216815F8010B4860E08C002858
:100B1000D5D14B4600224021204600F087F908B18C
:100B20000320DDE794F83900322805D084F83960D5
:100B300084F838700020D3E7222084F83900F7E7E2
:100B40000220CDE7144800B5026887B0002142F0CA
:100B500080020260026802F080020592026842F0A0
:100B600008020260026802F008020592026842F080
:100B700004020260006800F0040005904FF4805009
:100B800000900120CDE90101039169460348FFF778
:100B90007BFB07B000BD000030380240000C024073
:100BA0000848074901604FF4E1314160002181604C
:100BB0000C22C160C0E904128161C161FFF709BF65
:100BC00000480040D03D00200907090E002806DA41
:100BD00000F00F0000F1E02080F8141D704700F1D4
:100BE000E02080F80014704710B5FFF739FCBDE82D
:100BF0001040FFF7EABE0000184800B502688DB04B
:100C0000002142F080520260006800F080500C9099
:100C10001348026842F4804202600068069100F4C2
:100C200080400C900220009001200390102004903E
:100C30006846FFF71DFDFFF79BFC4FF47A71B0FB90
:100C4000F1F0FFF7AEFE0420FFF79EFE00221146F2
:100C5000501EFFF75BFC0DB000BD000040380240A5
:100C6000007000401048016841F4700101600F48B5
:100C7000016841F0010101600C4A00210832116055
:100C800002680B4B1A400260031D0A4A1A60026890
:100C900022F48022026005480C30016002495806A7
:100CA000803908607047000088ED00E0003802409D
:100CB000FFFFF6FE103000242DE9F04104460068E5
:100CC0000169E26821F440510A4302612068C16869
:100CD00049F20C6291432369A268E5691A4363698A
:100CE0002B431A430A43C2602068416921F44072D1
:100CF000A16911434161E06964263225B0F5004FD6
:100D0000484A494920681DD0884201D0904269D1A3
:100D1000FFF75EFC00EBC00101EB00106168B0461C
:100D20008900B0FBF1F1B1FBF8F6FFF751FC00EBE5
:100D3000C00101EB001061688900B0FBF1F7FFF71B
:100D400047FC68E0884201D0904219D1FFF740FC8F
:100D500000EBC00101EB00106168B0464900B0FB38
:100D6000F1F1B1FBF8F6FFF733FC00EBC00101EB4A
:100D7000001061684900B0FBF1F7FFF729FC18E0AB
:100D8000FFF710FC00EBC00101EB00106168B046FA
:100D90004900B0FBF1F1B1FBF8F6FFF703FC00EB03
:100DA000C00101EB001061684900B0FBF1F7FFF7EB
:100DB000F9FB00EBC00101EB001061684900B0FBDA
:100DC000F1F1B1FBF8F06FF01801484307EB800038
:100DD00005EB0011B1FBF8F0216866F31F10886085
:100DE000BDE8F081FFF7DEFB00EBC00101EB001076
:100DF0006168B0468900B0FBF1F1B1FBF8F6FFF78E
:100E0000D1FB00EBC00101EB001061688900B0FB71
:100E1000F1F7FFF7C7FB00EBC00101EB00106168C1
:100E20008900CCE700140140001001402DE9F04793
:100E30001D4690460F460446FFF70CFB06465FEA48
:100E400008004FF000094FF0010808D030E0681C9E
:100E500005D095B1FFF7FEFA801BA8420DD8206897
:100E6000006837EA0000F2D127E0681C20D025B1E5
:100E7000FFF7F0FA801BA8421AD92068C16821F058
:100E80008001C1602068C16821F02001C160206834
:100E9000C16821F48071C1602068416921F00101BD
:100EA000416184F8398084F838900320BDE8F087E8
:100EB0002068006837EA0000D7D00020F6E700007D
:100EC0000FB4054B10B503A9044A029800F018F8B6
:100ED00010BC5DF814FB0000C11101080C000020DB
:100EE00002E008C8121F08C1002AFAD170477047F3
:100EF000002001E001C1121F002AFBD17047000051
:100F00002DE9FF4F8DB09B460F460446002606E0B4
:100F100025280BD05A460F999047641C761C2078E0
:100F20000028F5D111B03046BDE8F08F0025A84665
:100F30000122984900E0054314F8013F203B02FAE2
:100F400003F00842F7D120782E2817D114F8010FAA
:100F500045F004052A280ED06FF02F022078A0F16A
:100F6000300109290AD808EB880102EB410100EBA6
:100F70000108641CF2E757F8048B641C20786C2885
:100F80000DD004DC4C2812D06A2811D104E074285A
:100F90000DD07A280CD10AE045F4001507E06178FD
:100FA00045F48015814202D1641C05F58015641C4E
:100FB0002278692A45D008DC002AB3D0582A69D0A3
:100FC000632A10D0642A08D13BE0702A67D0732AC4
:100FD00013D0752A5CD0782A5CD010465A460F99F7
:100FE0009047761CD3E017F8040B8DF80000002022
:100FF0008DF80100E946012003E057F8049B4FF00B
:10100000FF3069074FF0000501D40AE06D1C45452B
:101010000DDA8542FADB19F805100029F6D106E051
:101020006D1C8542FCDB19F805100029F8D12E440F
:1010300004E019F8010B5A460F9990476D1EF8D23B
:10104000A5E00A200021CDE90801C5F302500228DD
:101050000DD001CFC117031E71F100030DDA4FF05F
:10106000000CD0EB0C006CEB01012D2308E0FF1D00
:1010700027F00707F7E80201EDE72B0504D52B233E
:101080008DF8283001233BE0EB0739D02023F7E728
:101090000A2000E010200021CDE9080107E010201F
:1010A000002145F00405CDE908014FF00808C5F31B
:1010B000025002280FD001CF00214FF0000A2B0769
:1010C0001FD5702A0DD0DDE908C38CF0100C5CEA46
:1010D000030C0CD015E0FF1D27F00707F7E802010D
:1010E000EBE740228DF828204FF0010A0BE050EA90
:1010F000010306D030238DF828308DF829200223F3
:101100009A46582A04D024A20DF120090B9209E036
:1011100026A2F9E7DDE90823FFF752F80B9B9B5C59
:1011200009F8013D50EA0102F4D1ADEB090020308D
:101130000890680701D44FF001080899884502DD3E
:10114000A8EB010000E000208046002506E00AA888
:101150005A46405D0F9990476D1C761C5545F6DB4D
:1011600004E030205A460F999047761CB8F10001F0
:10117000A8F10108F5DC05E019F8010B5A460F99B2
:101180009047761C0899481E08900029F4DC641CDE
:10119000C5E60000092801003031323334353637D6
:1011A00038396162636465660000000030313233B3
:1011B0003435363738394142434445460000000053
:1011C00013B54FF6FF73012269460248FFF756FC3C
:1011D00000981CBDD03D0020FFF74AF9FFF70CFD39
:1011E000FFF7B0FCFFF7DCFC0BA0FFF769FE18A0CF
:1011F000FFF766FE08A0FFF763FE23492148086059
:1012000000F044F804A0FFF75BFE11A0FFF758FEC2
:1012100001A0FFF755FEF5E70A2D2D2D2D2D2D2DC3
:101220002D2D2D2D2D2D2D2D2D2D2D2D2D2D2D2DEE
:101230002D2D2D2D2D2D2D2D2D2D2D2D2D2D2D2DDE
:101240002D2D2D2D2D2D2D2D2D2D2D0A00000000A5
:101250000A202020202020202020202020202020A4
:10126000202053544D3332463420494150204150C0
:10127000503220202020202020202020202020202C
:1012800020200A000000010808ED00E02DE9F041EF
:101290000A4C00200A4E0B4D4FF47767206056F839
:1012A000201045F8201008A0FFF70AFE2068401C17
:1012B0002060B842F3DBBDE8F081000000000020B0
:1012C0000000010810000020307825782C0D0A005D
:1012D00000000000010203040102030406070809DC
:1012E000001301080000002010000000E00E0108BB
:1012F000101301081000002000420000F00E010849
:1013000000000000000000000024F40000000000C5
:040000050801018964
:00000001FF
